:020000040000FA
:0408000000EF2CF0E9
:0457FC0000000000A9
:10580000A0EF2FF000C0E5FF01C0E5FF00EE62F061
:1058100002EC2FF0006E00C0F3F000C0F4F002ECD8
:105820002FF0006E0001E96F00500001F42702EC38
:105830002FF0006E0001E86F00500001F42702EC29
:105840002FF0006E00C0F5F000500001F4270001B9
:10585000F551040A24E10001E951D8A4DBD0E85154
:10586000D8A4D8D00001F351020A01E0D3D002EC51
:105870002FF0006E0001EB6F00500001F42702ECE6
:105880002FF0006E0001EA6F00500001F42702ECD7
:105890002FF0006E0001F427F451D8A4B3D000011A
:1058A000F551010A20E102EC2FF0006E0001F4270F
:1058B000F451D8A4A7D00001F2B3BCEC2DF08BECCE
:1058C0002FF00001F2A50BD0C00E0001E46F570EBF
:1058D000E56FE66BE76BBCEC2DF08BEC2FF0590E0F
:1058E00070EC2FF09AD00001EB510001E71914E1A0
:1058F0000001EA510001E6190FE10001E951000140
:10590000E5190AE1C00E0001E815006EC00E0001A5
:10591000E415016E00180FE00001F2A302D0BCEC08
:105920002DF08BEC2FF0E8C0E4F0E9C0E5F0EAC020
:10593000E6F0EBC0E7F00001F551040A01E15ED0AA
:105940000001F551D8A462D00001F351D8B456D06B
:105950000001EB51D8A45AD0EA51E00BD8A456D09C
:105960000001F2A912D00001F3514AEC2EF0400ED2
:1059700096EC2FF00001E9514AEC2EF00001E851BD
:105980004AEC2EF0200E96EC2FF0EAC0F8FFE9C0AA
:10599000F7FFE8C0F6FF000100EE6AF022EE00F02B
:1059A000E8513F0BD926D8B0DA2ADD5202EC2FF0AD
:1059B0000001F427DC6E0900F55C05E00001F283CC
:1059C0002A0E96EC2FF00001F2A906D0DF504AEC27
:1059D0002EF0200E96EC2FF00001F32FE7D702EC0B
:1059E0002FF0006E0001F427F45108E00001E46993
:1059F000E569E669E7690001F29304D0580E70EC9E
:105A00002FF00BD07A0E70EC2FF007D0750E70ECE3
:105A10002FF003D06C0E70EC2FF0E4CF01F0E4CF48
:105A200000F01200FF0E926E936E946E956E966E5D
:105A3000970ED56E8A909390B06A2F0EAF6EB8868F
:105A4000AC8AAC84AC8CAC90AB8CAB8E0001E46BBC
:105A5000E56BE66BE76B0001E86BE96BEA6BEB6B00
:105A60008BEC2FF00001F26B93988A888A80AB98B8
:105A70004B0E96EC2FF0AAEC2FF00001EC6BED6BC7
:105A8000006A8AB0002A0050010A02E1AAEC2FF055
:105A90000001606BC2EC2EF000016051D8B45CD004
:105AA0008A80AB988AA802D08A9801D08A8861C07F
:105AB00000F00050520A03E161EC2FF00BD00050CF
:105AC000500A03E152EC2FF005D00050560A02E1D3
:105AD0007EEC2EF00001F2A13FD00050450A03E118
:105AE00040EC2FF039D000503A0A03E102EC2CF0E0
:105AF00033D00050720A03E1A1EC2EF02DD00050FB
:105B0000410A03E1CBEC2FF027D00050760A24E1C4
:105B1000006A00016251300A01E1002A0050D88079
:105B2000E866D890006A00360050010BE838E8407B
:105B3000F46E0001F251F70BF410F26F320E000117
:105B4000625D006A00360050010BE838F46E000117
:105B5000F251EF0BF410F26F0001F2B191D7000196
:105B6000ED51800F800F02E1A10EEC5DD8A088D727
:105B7000CBEC2FF085D7120000C0E5FF01C0E5FF98
:105B800002C0E5FF03C0E5FF0001E4513F0B04E064
:105B9000210E96EC2FF075D00001E75103E1E6519C
:105BA000E00BD8A46ED0580E0001E55D02E1000EB6
:105BB000E45D01E366D0E4C000F0E5C001F0E6C0BA
:105BC00002F0E7C003F0005007E10150080A04E1C9
:105BD000025002E1035001E013D000C2E0F001C224
:105BE000E1F002C2E2F003C2E3F00201006BEF0E4B
:105BF000016F2C0E026FF00E036F0001F28515D0BD
:105C00000050C00A07E10150570A04E1025002E1C6
:105C1000035001E00AD0E0C03CF2E1C03DF2E2C036
:105C20003EF2E3C03FF20001F2950001F2A70BD073
:105C3000200E96EC2FF00001E5514AEC2EF0000109
:105C4000E4514AEC2EF0E6C0F8FFE5C0F7FFE4C0EF
:105C5000F6FF940EB2EC2FF00A0002EE00F0000105
:105C6000080EEE6F080EEF6FEE50F56E0F00EF2F7F
:105C7000FBD7840E77D9EE2FF5D7A694570E70EC8C
:105C80002FF0E4CF03F0E4CF02F0E4CF01F0E4CF53
:105C900000F0120000C0E5FF01C0E5FF02C0E5FF13
:105CA000006E00380F0B026E300E02260250016E9D
:105CB0003A0E015C06E30150026E070E0226025006
:105CC000016E015096EC2FF00F0E0014006E300E96
:105CD00000260050016E3A0E015C06E30150006E92
:105CE000070E00260050016E015096EC2FF0E4CF15
:105CF00002F0E4CF01F0E4CF00F0120000EE62F019
:105D0000000160050001EF6FEF07010EEE6FEE512D
:105D1000C5EC2FF004E10A0EEE6FC5EC2FF0EE5C3F
:105D2000D8A41200EE2BEF2FF2D7EE51C5EC2FF0D6
:105D3000D8A41200560E70EC2FF00001F281F295FB
:105D4000120000C0E5FF00EE62F002EC2FF0F76EEB
:105D500002EC2FF0F66E720E96EC2FF0200E96EC01
:105D60002FF0100E006E0900F5504AEC2EF0200EB8
:105D700096EC2FF0002EF7D70A0E96EC2FF0E4CF1A
:105D800000F01200BFEC2FF0000100EE60F0E2EC3A
:105D90002EF0E86614D0AE50EE6EEE6FEF6FD8B412
:105DA0000ED0BFEC2FF0E2EC2EF0E86608D0AE503B
:105DB000EE6EEF27EE2FF5D7EF53D8B412000001A7
:105DC000606B12009EBA08D0F2A4FCD70001EC2B45
:105DD00001E3ED2BE86815D08A98ABB202D0ABA4F2
:105DE00004D0AAEC2FF0E8680CD0ABA009D0AE50DC
:105DF00005E1BFEC2FF0E2EC2EF003D0CBEC2FF05E
:105E0000E86A12000001EECFEEF0EECFEFF0D00E18
:105E1000EE27EF27F60EEE25F90ED8B0EE27F60E98
:105E2000EF25F90ED8B0EF27EE39EF25E850120034
:105E300000EE68F000016051F80F0001EE6F09E01C
:105E4000F05D07E3EE50A86E7FEC2FF0A92AEE2F4D
:105E5000F9D7A86A7FEC2FF0120000C0E5FF01C05F
:105E6000E5FF006A00EE62F0060E016EEE500026BD
:105E7000012EFCD70050E4CF01F0E4CF00F0120077
:105E800000EE61F0000160510001EE6F07E0EE07E7
:105E900005E0EE5096EC2FF0EE2FFBD70A0E96ECB5
:105EA0002FF012002DEC2FF0B80A0AE1010EA96EB6
:105EB000080E0001F06F18EC2FF0500E70EC2FF070
:105EC00012002DEC2FF0A00A0AE10A0EA96E100EA6
:105ED0000001F06F18EC2FF0520E70EC2FF0120052
:105EE00000C0E5FF006E200E96EC2FF0005096ECFF
:105EF0002FF00A0E96EC2FF0E4CF00F01200A69ED1
:105F0000A69CA684550EA76EAA0EA76EA682A6B260
:105F1000FED7A69412000001F2930001400EEE6F2E
:105F200002EE00F0EE68EE2FFDD7120000C0E5FF94
:105F3000006E9EA8FED700C0ADFFE4CF00F01200B7
:105F400011EEFFF021EEFFF0F86AA68EA69C12EC8F
:105F50002DF0FFD7ACA2FED78A90AE50AE50AB98D2
:105F6000AB881200A66E550EA76EAA0EA76EA6826B
:105F70001200BBEF2FF012EC2DF0BDEF2FF0FE0E54
:105F8000D76E120ED66EF2941200A96EA69CA69E33
:0A5F9000A680A8501200FEEF2BF0CF
:020000040030CA
:0E000000E03EDAE0FF7D9AFFFFFFFFFFFFFF0B
:0200000400F00A
:0400000000000000FC
:00000001FF
